:060000000A128A11E42F30
:10000C0083120313C6006E304602031CE42803302F
:10001C00BA003A08A4000A30F7000030F80046088D
:10002C00BB00BC013B08F2003C08F3006430F0005C
:10003C000030F1000A168A1130210A128A11710857
:10004C00FA007008F9000A168A11C7210A128A11DF
:10005C007708093E0A168A11A9200A128A11503E05
:10006C0084000A168A110A200A128A1183120313B9
:10007C00A7000A168A110A200A128A11A8000A1669
:10008C008A110A200A128A11A9000330BD003D080A
:10009C00A4006430F7000030F8004608BE00BF0131
:1000AC003E08F9003F08FA000A168A11C7210A1205
:1000BC008A117708123E0A168A11A9200A128A118F
:1000CC00503E84000A168A110A200A128A118312E1
:1000DC000313AA000A168A110A200A128A11AB000D
:1000EC000A168A110A200A128A11AC000A168A1101
:1000FC0050250A128A11831203132708C3002808FB
:10010C00C4002908C5000330BA003A08A400460808
:10011C00BB00BC013B08F2003C08F3000A30F000C5
:10012C000030F1000A168A1130210A128A11700867
:10013C000A168A11A9200A128A11503E84000A1646
:10014C008A110A200A128A1183120313A7000A16B5
:10015C008A110A200A128A11A8000A168A110A208A
:10016C000A128A11A9004308AA004408AB004508EA
:10017C00AC000A168A1150250A128A118312031335
:10018C002708C0002808C1002908C2000030A700B9
:10019C000030A8003F30A9004008AA004108AB007D
:1001AC004208AC000A168A11502583120313270843
:1001BC00B7002808B8002908B90008000B3046021F
:1001CC00031C6E290330BA003A08A4004608BB0091
:1001DC00BC013B08F2003C08F3000A30F000003090
:1001EC00F1000A168A1130210A128A1170080A16B7
:1001FC008A11A9200A128A11503E84000A168A110B
:10020C000A200A128A1183120313A7000A168A11F4
:10021C000A200A128A11A8000A168A110A200A1248
:10022C008A11A9000330BD003D08A4000A30F70074
:10023C000030F8004608BE00BF013E08F9003F0838
:10024C00FA000A168A11C7210A128A117708093E88
:10025C000A168A11A9200A128A11503E84000A1625
:10026C008A110A200A128A1183120313AA000A1691
:10027C008A110A200A128A11AB000A168A110A2066
:10028C000A128A11AC000A168A1150250A128A1118
:10029C00831203132708C3002808C4002908C500CB
:1002AC000030A7000030A8003F30A9004308AA0086
:1002BC004408AB004508AC000A168A11502583127D
:1002CC0003132708B7002808B8002908B90008004C
:1002DC000030A7000030A8003F30A9000330BA005E
:1002EC003A08A40046080A168A11A9200A128A1193
:1002FC00503E84000A168A110A200A128A118312AF
:10030C000313AA000A168A110A200A128A11AB00DA
:10031C000A168A110A200A128A11AC000A168A11CE
:10032C005025831203132708B7002808B8002908A2
:10033C00B900080083160313D2005B308312031339
:10034C00DE005E0883160313C50001308312DA0742
:10035C00FF305A0784000A168A110A200A128A11E1
:10036C00DE005E0883160313D80058080319DF2F2C
:10037C00253058060319C629580883120313CE2FAB
:10038C00C601C701831203135A0884000A168A1186
:10039C000A200A128A112E3A031D242A83160313EB
:1003AC004717013083120313DE005E08DA07831649
:1003BC000313D301D40183125A0884000A168A113C
:1003CC000A200A128A110A168A15B4260A128A11F0
:1003DC00031C2C2A831603135408F1005308F00055
:1003EC000A30F2000030F3000A168A1539270A1277
:1003FC008A11831203135A0884000A168A110A20E0
:10040C000A128A117007DE000030031801307107E0
:10041C00DF005E08D03E83160313D3008312031350
:10042C005F080318013EFF3E83160313D40001300E
:10043C0083120313DE005E08DA07E1298316031327
:10044C00D301D40147162C2A4715422A01308312B6
:10045C000313DA07FF305A0784000A168A110A20A0
:10046C000A128A1183160313D800003A0319DF2FDE
:10047C00663A03192A2AAB29003046058312031366
:10048C00DE00073083160313470583120313DF00C6
:10049C005E085F040319612F83160313471E5A2A43
:1004AC000630D3000030D4004508840083130008C4
:1004BC00D500840A0008D600840A0008D70003304F
:1004CC0083120313DE005E0883160313C507550859
:1004DC00F0005608F1005708F2000030F30000302D
:1004EC00F4000030F5000A168A1122220A128A1131
:1004FC000318992A831603135508F0005608F100C7
:10050C005708F2000A168A15A4260A128A117008D6
:10051C0083160313D5007108D6007208D700033078
:10052C00C6040030C70483160313CC01CD01570851
:10053C005604550403198D2BD53084008313000801
:10054C0083120313DE00840A0008DF00840A00080B
:10055C00E000840A0008E1000F300310E10CE00C0D
:10056C00DF0CDE0CFF3E031DB32AFF305E05E200FC
:10057C0000305F05E3006208823E83160313CC0053
:10058C008312031363080318013EFF3E8316031303
:10059C00CD00FF30CC070318CD0AFF30CD07033058
:1005AC00F0000030F1004D08F3004C08F2000A1680
:1005BC008A1539270A128A11710883160313CD0084
:1005CC007008CC000A30F7000030F8004D08FA0033
:1005DC004C08F9000A168A11C7210A128A117808E8
:1005EC0083160313CD007708CC00CD1F032BFF30EF
:1005FC00CC070318CD0AFF30CD074C03FF3A0A1283
:10060C008A1573210A128A11831203133708831671
:10061C000313CE0083120313380883160313CF0081
:10062C0083120313390883160313D0005508831261
:10063C000313A70083160313560883120313A80091
:10064C0083160313570883120313A900831603138D
:10065C004E0883120313AA00831603134F08831248
:10066C000313AB0083160313500883120313AC005F
:10067C000A168A1150250A128A11831203132708AD
:10068C0083160313CE008312031328088316031357
:10069C00CF0083120313290883160313D0004E08CE
:1006AC00F0004F08F1005008F2000030F3008030E9
:1006BC00F4003F30F5000A168A1122220A128A1120
:1006CC000318702BFF3083160313CC070318CD0AC5
:1006DC00FF308C2B831603134E08F0004F08F100EB
:1006EC005008F2000030F3002030F4004130F500E7
:1006FC000A168A1122220A128A11031C8D2B013030
:10070C0083160313CC070318CD0A0030CD078316CC
:10071C0003135408803AFF0080307F02031D982B8E
:10072C000D3053020318D32B8316031353080A12EC
:10073C008A1106200A128A11831203133708C70084
:10074C003808C8003908C9008316031355088312EA
:10075C000313CA0083160313560883120313CB002A
:10076C0083160313570883120313CC000A168A113D
:10077C00F7260A128A1183120313470883160313F0
:10078C00D50083120313480883160313D600831273
:10079C000313490883160313D700831603134D085C
:1007AC00803AFF0080307F02031DDE2B0A304C02A2
:1007BC000318112C831603135708560455040319F8
:1007CC006A2C550883120313C000831603135608B2
:1007DC0083120313C10083160313570883120313E8
:1007EC00C2000A168A1149230A128A1183120313B2
:1007FC004308420441044004031D6A2C831603136E
:10080C004D08803AFF0080307F02031D0F2C023010
:10081C004C02031C6A2C831603134E08F0004F087D
:10082C00F1005008F2007030F3008930F4004030D1
:10083C00F5000A168A1122220A128A110318282C92
:10084C00F730292CF83083160313CC070318CD0A84
:10085C00FF30CD074C080A128A1573210A128A112F
:10086C0083120313370883160313CE00831203136A
:10087C00380883160313CF00831203133908831629
:10088C000313D0005508F0005608F1005708F20089
:10089C004E08F3004F08F4005008F5000A168A11B0
:1008AC008D240A128A11730883160313CB00720865
:1008BC00CA007108C9007008C8000030D5000030AB
:1008CC00D6000030D700D92C831603135508831299
:1008DC000313C00083160313560883120313C100BD
:1008EC0083160313570883120313C2000A168A11C6
:1008FC0049230A128A118312031343088316031324
:10090C00CB0083120313420883160313CA0083120D
:10091C000313410883160313C90083120313400801
:10092C0083160313C8004B08FB004A08FA00490859
:10093C00F9004808F8000A168A15D5270A128A11F8
:10094C00780883120313D4007908D5007A08D600EE
:10095C0083160313550883120313D700831603134E
:10096C00560883120313D8008316031357088312F7
:10097C000313D9000A168A1518270A128A11831232
:10098C000313540883160313D5008312031355085D
:10099C0083160313D600831203135608831603130E
:1009AC00D700CC01CD01D801D80A0A30580603195A
:1009BC002F2D580883120313DE0001300310DE0DB7
:1009CC00FF3E031DE42C03105E0D013E84000A164D
:1009DC008A110A200A128A11DF000A168A110A20CB
:1009EC000A128A11E0000A168A110A200A128A11C8
:1009FC00E1000A168A110A200A128A11E200620822
:100A0C00831603134B02031D212D8312031361085C
:100A1C00831603134A02031D212D8312031360084E
:100A2C00831603134902031D212D831203135F0840
:100A3C00831603134802031C2F2D0130831203135A
:100A4C00DE005E0883160313D8070A305806031D10
:100A5C00DF2C0330460583120313DE0000308316AF
:100A6C000313470583120313DF005E085F040319A9
:100A7C00502D2D30DE008316031352088400831290
:100A8C0003135E08831780000130DE005E088316B6
:100A9C000313D207FF308312DE005E0883160313A4
:100AAC00D807580A0319D62D580883120313DE00F1
:100ABC0001300310DE0DFF3E031D5F2D03105E0D94
:100ACC00013E84000A168A110A200A128A11F000CB
:100ADC000A168A110A200A128A11F1000A168A11C2
:100AEC000A200A128A11F2000A168A110A200A1226
:100AFC008A11F300831603134B08F7004A08F6001B
:100B0C004908F5004808F4000A168A117F220A12D7
:100B1C008A11730883160313D1007208D000710870
:100B2C00CF007008CE000030F3000030F20000302F
:100B3C00F1000A30F0005108F7005008F6004F0899
:100B4C00F5004E08F4000A168A117B210A128A114C
:100B5C00730883160313D1007208D0007108CF00FC
:100B6C007008CE004E08303E83120313402D3030F7
:100B7C0083120313DE0083160313520884008312BE
:100B8C0003135E08831780000130DE005E088316B5
:100B9C000313D207FF30CC070318CD0AFF30CD0763
:100BAC004D08803AFF0080307F02031DDF2D01309D
:100BBC004C020318BD2D831603135408803AFF0012
:100BCC0080307F02031DEC2D09305302031CF02DE5
:100BDC000830F32D83160313530883120313DE001E
:100BEC005E0883160313D800580883120313DE0023
:100BFC00DF01DE1BDF035E0883160313D3028312AF
:100C0C0003135F0883160313031CD403D402580880
:100C1C000319232E2E3083120313DE0083160313C5
:100C2C0052088400831203135E088317800001307E
:100C3C00DE005E0883160313D20758080A128A15C1
:100C4C0073210A128A1183120313370883160313B4
:100C5C00C20083120313380883160313C3008312D4
:100C6C000313390883160313C400420883120313B9
:100C7C00AA0083160313430883120313AB008316D5
:100C8C000313440883120313AC0083160313550893
:100C9C0083120313A700831603135608831203133E
:100CAC00A80083160313570883120313A9000A160E
:100CBC008A1150250A128A11831203132708C000C7
:100CCC002808C1002908C2000A168A1149230A12F1
:100CDC008A1183120313430883160313CB00831268
:100CEC000313420883160313CA008312031341082B
:100CFC0083160313C90083120313400883160313CE
:100D0C00C800FF3083120313DE005E088316031342
:100D1C00D807580A03195C2F580883120313DE00F6
:100D2C0001300310DE0DFF3E031D972E03105E0DE8
:100D3C00013E84000A168A110A200A128A11F00058
:100D4C000A168A110A200A128A11F1000A168A114F
:100D5C000A200A128A11F2000A168A110A200A12B3
:100D6C008A11F300831603134B08F7004A08F600A8
:100D7C004908F5004808F4000A168A117F220A1265
:100D8C008A11730883160313D1007208D0007108FE
:100D9C00CF007008CE000030F3000030F2000030BD
:100DAC00F1000A30F0005108F7005008F6004F0827
:100DBC00F5004E08F4000A168A117B210A128A11DA
:100DCC00730883160313D1007208D0007108CF008A
:100DDC007008CE004E08303E83120313DE008316DB
:100DEC00031352088400831203135E0883178000D8
:100DFC000130DE005E0883160313D20758088312F5
:100E0C000313DE0001300310DE0DFF3E031D092F1E
:100E1C0003105E0D013E84000A168A110A200A1284
:100E2C008A11F0000A168A110A200A128A11F1009E
:100E3C000A168A110A200A128A11F2000A168A115D
:100E4C000A200A128A11F300831603134B08F700C9
:100E5C004A08F6004908F5004808F4000A168A11F9
:100E6C007B210A128A11730883160313CB007208B4
:100E7C00CA007108C9007008862E30308312031323
:100E8C00DE008316031352088400831203135E08DA
:100E9C00831780000130DE005E0883160313D2072F
:100EAC00FF30D3070318D40AFF30D4075308540477
:100EBC000319AB29432F8316031353085404031D42
:100ECC00732F4B084A0449044804031D732F013047
:100EDC00D3070318D40A0030D4075808831203131D
:100EEC00DE00DF01DE1BDF035F08803AE0008316C3
:100EFC0003135408803A831203136002031D8C2FD2
:100F0C00831603135308831203135E020318992FDD
:100F1C0083160313530883120313DE005E08831633
:100F2C000313D800BB2F8316031358088312031323
:100F3C00DE00DF01DE1BDF03831603135408803A47
:100F4C0083120313E0005F08803A6002031DB22F86
:100F5C005E088316031353020318BB2F8316031367
:100F6C005808D300D401D31BD403033083160313C6
:100F7C00460583120313DE00003083160313470566
:100F8C0083120313DF005E085F040319AB292D30B5
:100F9C00DE008316031352088400831203135E08C9
:100FAC00831780000130DE005E0883160313D2071E
:100FBC00AB29520884008317800108008313673023
:100FCC00840070300A168A15AC260A128A11A030D9
:100FDC008400C2300A168A15AC260A128A118317AD
:100FEC0090308400AE300A168A15AC2683010A12A2
:040FFC008A150E2C18
:10100200F90100300A168A155A270A128A15831224
:10101200031307138830F0001330F1000A168A1503
:10102200D0260A128A15F9010330790203183028F2
:1010320038300A168A155A270A128A156430F000C7
:101042000030F1000A168A15D0260A128A150130DC
:10105200F8007808F90703307902031C19280C30CC
:101062000A168A155A270A128A1501300A168A1593
:101072005A270A128A1506300A168A155A270800B4
:10108200703084000008F600840A0008F700840A21
:101092000008F800840A0008F9000310780D790DA1
:1010A200FA007A0883120313A5002508031D62289B
:1010B2000030F3000030F2000030F1000030F000A8
:1010C2000800733084000008F600840A0008F70064
:1010D200840A0008F800840A0008F9000310780D59
:1010E200790DFA007A08A4002408031D8128003033
:1010F200F3000030F2000030F1000030F000080090
:101102007030840000308004840A00308004840A35
:1011120080308004840A0030800470308400FF3004
:101122008005840AFF308005840AFF308005840A26
:10113200003080057330840000308004840A00305F
:101142008004840A80308004840A00308004733072
:101152008400FF308005840AFF308005840AFF3056
:101162008005840A003080050030A3000030A20010
:101172000030A1000030A0007F30A502A03024077B
:10118200F6007608A5022030F6007608A4000130A9
:10119200F6000310A00DA10DA20DA30DF60BCA2897
:1011A200733084000008F600840A0008F700840AFD
:1011B2000008F800840A0008F90070308400000872
:1011C200FA00840A0008FB00840A0008FC00840A72
:1011D2000008FD0079087D02031DF92878087C02C9
:1011E200031DF92877087B02031DF92876087A0285
:1011F200031C1E29733084000008F600840A0008CC
:10120200F700840A0008F800840A0008F900703028
:10121200840076088002840A7708031C770F800214
:10122200840A7808031C780F8002840A7908031C58
:10123200790A800203308402201470308400031083
:10124200800D840A800D840A800D840A800D840337
:10125200840384030130A402031DC828A51F4F295B
:101262002508803A9F3E03183F290030F3000030E2
:10127200F2000030F1000030F000080001300310ED
:10128200A30CA20CA10CA00CFF3E031D40290130AF
:10129200F6007608A50703196A293F29203025029E
:1012A200031C67290030F3000030F2000030F10027
:1012B2000030F00008000130F6000310A00DA10D6F
:1012C200A20DA30DF60B5E290130A5022508031D10
:1012D2005C292308F3002208F2002108F10020080B
:1012E200F000080083120313BF00BF1FC42ABF0906
:1012F200BF0A3F08803A123E031C372A0330BA0065
:101302003A08A4000A30F7000030F8003F08F20063
:10131200F301F21BF3036430F0000030F1000A160F
:101322008A1130210A128A157108FA007008F90030
:101332000A168A11C7210A128A157708093E0A1667
:101342008A11A9200A128A15503E84000A168A11AF
:101352000A200A128A1583120313A7000A168A1199
:101362000A200A128A15A8000A168A110A200A12ED
:101372008A15A9000330BB003B08A4006430F700C3
:101382000030F8003F08F900FA01F91BFA030A16C7
:101392008A11C7210A128A157708123E0A168A1183
:1013A200A9200A128A15503E84000A168A110A20C0
:1013B2000A128A1583120313AA000A168A110A2036
:1013C2000A128A15AB000A168A110A200A128A1515
:1013D200AC000A168A1150250A128A1583120313C9
:1013E2002708BC002808BD002908BE000330BA0047
:1013F2003A08A4003F08F200F301F21BF3030A309B
:10140200F0000030F1000A168A1130210A128A1502
:1014120070080A168A11A9200A128A15503E840001
:101422000A168A110A200A128A1583120313A700C8
:101432000A168A110A200A128A15A8000A168A11A7
:101442000A200A128A15A9003C08AA003D08AB002E
:101452003E08AC000A168A1150258312031327088E
:10146200B7002808B8002908B90008003F08803AE8
:10147200753E031CA52A0330BA003A08A4003F08AF
:10148200F200F301F21BF3030A30F0000030F10026
:101492000A168A1130210A128A1570080A168A1150
:1014A200A9200A128A15503E84000A168A110A20BF
:1014B2000A128A1583120313A7000A168A110A2038
:1014C2000A128A15A8000A168A110A200A128A1517
:1014D200A9000330BB003B08A4000A30F70000302B
:1014E200F8003F08F900FA01F91BFA030A168A11FB
:1014F200C7210A128A157708093E0A168A11A920FD
:101502000A128A15503E84000A168A110A200A120B
:101512008A1583120313AA000A168A110A200A12D4
:101522008A15AB000A168A110A200A128A15AC0023
:101532000A168A115025831203132708B7002808B8
:10154200B8002908B90008000330BA003A08A4001C
:101552003F080A168A11A9200A128A15503E8400F1
:101562000A168A110A200A128A1583120313B70077
:101572000A168A110A200A128A15B8000A168A1156
:101582000A20B90008003F08803A123E031C812B52
:101592000330BA003A08A4000A30F7000030F8001D
:1015A2003F08F200F301F21BF3036430F000003055
:1015B200F1000A168A1130210A128A157108FA00FE
:1015C2007008F9000A168A11C7210A128A157708CB
:1015D200093E0A168A11A9200A128A15293E840098
:1015E2000A168A110A200A128A1583120313A70007
:1015F2000A168A110A200A128A15A8000A168A11E6
:101602000A200A128A15A9000330BB003B08A40075
:101612006430F7000030F8003F08F900FA01F91BC6
:10162200FA030A168A11C7210A128A157708123E8E
:101632000A168A11A9200A128A15293E84000A165E
:101642008A110A200A128A1583120313AA000A16A3
:101652008A110A200A128A15AB000A168A110A2078
:101662000A128A15AC000A168A1150250A128A1526
:10167200831203132708BC002808BD002908BE00F6
:101682000330BA003A08A4003F08F200F301F21B4B
:10169200F3030A30F0000030F1000A168A113021FB
:1016A2000A128A1570080A168A11A9200A128A15C6
:1016B200293E84000A168A110A200A128A15831208
:1016C2000313A7000A168A110A200A128A15A80013
:1016D2000A168A110A200A128A15A9003C08AA00D1
:1016E2003D08AB003E08AC000A168A115025831251
:1016F20003132708B7002808B8002908B900080012
:101702003F08803A753E031CEF2B0330BA003A08BB
:10171200A4003F08F200F301F21BF3030A30F000C9
:101722000030F1000A168A1130210A128A15700857
:101732000A168A11A9200A128A15293E84000A165D
:101742008A110A200A128A1583120313A7000A16A5
:101752008A110A200A128A15A8000A168A110A207A
:101762000A128A15A9000330BB003B08A4000A3004
:10177200F7000030F8003F08F900FA01F91BFA03FC
:101782000A168A11C7210A128A157708093E0A1613
:101792008A11A9200A128A15293E84000A168A1182
:1017A2000A200A128A1583120313AA000A168A1142
:1017B2000A200A128A15AB000A168A110A200A1296
:1017C2008A15AC000A168A115025831203132708C2
:1017D200B7002808B8002908B90008000330BA0089
:1017E2003A08A4003F080A168A11A9200A128A158B
:1017F200293E84000A168A110A200A128A158312C7
:101802000313B7000A168A110A200A128A15B800B1
:101812000A168A110A20B90008000A168A15E62655
:101822000A128A15FA01FA0A8730FB008030FC009E
:1018320002300A168A11F4200A128A15831203133F
:10184200E501E601FF306602DC3003196502031888
:10185200372C0130E5070318E60A0030E607FF30AF
:101862006602DC3003196502031C2A2C0A168A154B
:101872009F260A128A15F801F80A00300A168A1100
:10188200BC200A128A153E300A168A1582270A12CD
:101892008A1583120313E8016808031DB92C0A167E
:1018A2008A15AA270A128A1583120313E400640810
:1018B200E8004D2CEC01EC0A3130B52C0230E4008A
:1018C2006408EC003230B52C0330E4006408EC000C
:1018D2003330B52C2B30E4006408EC002B30B52CEF
:1018E2000430E4006408EC003430B52C0530E40028
:1018F2006408EC003530B52C0630E4006408EC00D6
:101902003630B52C2D30E4006408EC002D30B52CB7
:101912000730E4006408EC003730B52C0830E400EE
:101922006408EC003830B52C0930E4006408EC009F
:101932003930B52C7830E4006408EC007830B52CEE
:101942002A30E4006408EC002A30B52CEC01303077
:10195200B52C2330E4006408EC002330B52C2F3082
:10196200E4006408EC002F30E4006408E800EB2C8B
:101972006808013A03195B2C033A03195F2C013AF8
:101982000319652C073A03196B2C013A0319712CC0
:10199200033A0319772C013A03197D2C0F3A0319E4
:1019A200832C013A0319892C033A03198F2C013A2B
:1019B2000319952C073A03199B2C013A0319A12C00
:1019C200033A0319A72C013A0319AA2C1F3A031947
:1019D200B02CEB2C6C030319102D02306C0603198A
:1019E200102D03306C060319102D04306C060319F8
:1019F200102D05306C060319102D06306C060319E4
:101A0200102D07306C060319102D08306C060319CF
:101A1200102D09306C06031D6C08031D462D67034B
:101A2200031D462DE701EA0114306A020318262D30
:101A32006A08A03E8400831380010130E400640838
:101A4200EA0714306A02031C192DFA01FA0A7730E8
:101A5200FB008030FC0001300A168A11F4200A12C1
:101A62008A15023083120313E4006408FA00773007
:101A7200FB008030FC0001300A168A11F4200A12A1
:101A82008A1583120313EA01492D6708031D522D9B
:101A92006C08E4006A08A03E840064088313800096
:101AA2005E2D23306C06031D5E2D6703031D5E2D24
:101AB200E70183160313BD01BD0A2B3083126806AA
:101AC2000319EB012D306806031D692DEB01EB0AAA
:101AD20078306806031D712D0230E4006408EB00C3
:101AE2002F306806031D792D0330E4006408EB00F3
:101AF2002A306806031D812D83160313BD01BD0A1A
:101B0200233083126806031D8A2D83160313BE0138
:101B1200BE0A83126A08A03E8400233083130006A3
:101B2200031D9E2DF801F80A6A08023E0A168A1160
:101B3200BC200A128A153D30AC2DF801F80A831236
:101B420003136A08023E0A168A11BC200A128A1579
:101B52008312031368080A168A1582270A128A1545
:101B6200831603133E03031DC12FBE018312031309
:101B7200EA010030ED000030EE000030EF00032EED
:101B82000030A7002030A8004130A9006D08AA004B
:101B92006E08AB006F08AC000A168A1150250A12B3
:101BA2008A15831203132708ED002808EE0029087E
:101BB200EF006D08C7006E08C8006F08C9006A0808
:101BC200A03E8400831300080A168A15FC260A1216
:101BD2008A15780883120313CA007908CB007A08A1
:101BE200CC000A168A11F7260A128A1583120313E9
:101BF2004708ED004808EE004908EF000130E40014
:101C02006408EA076A08A03E84002B3083130006AA
:101C12000319272E6A08A03E84002D3000060319FE
:101C2200272E6A08A03E8400783000060319272E6A
:101C32006A08A03E84002F3000060319272E6A0886
:101C4200A03E840023300006031DC12D6A08A03E79
:101C5200840023300006031D3A2E0030831603133E
:101C6200BF000030C0000030C10083120313EB013B
:101C7200C42E6A08013EE4006408E9006908E40031
:101C82006408EA00003083160313BF000030C0006E
:101C92000030C10083126A08A03E840023308313FF
:101CA20000060319C42E00308312A7002030A800BA
:101CB2004130A900831603133F0883120313AA00BD
:101CC20083160313400883120313AB008316031316
:101CD200410883120313AC000A168A1150250A1216
:101CE2008A1583120313270883160313BF00831276
:101CF2000313280883160313C00083120313290851
:101D020083160313C1003F0883120313C70083160F
:101D12000313400883120313C800831603134108F8
:101D220083120313C9006A08A03E840083130008CB
:101D32000A168A15FC260A128A15780883120313DA
:101D4200CA007908CB007A08CC000A168A11F72655
:101D52000A128A1583120313470883160313BF005E
:101D620083120313480883160313C000831203135C
:101D7200490883160313C100013083120313E400E0
:101D82006408EA074B2E003083160313B4000030B8
:101D9200B5000030B600831203136B08031DE92E51
:101DA200831603133F0883120313C700831603131A
:101DB200400883120313C8008316031341088312D9
:101DC2000313C9006D08CA006E08CB006F08072F05
:101DD20083126B03031D1D2F6D08C7006E08C80018
:101DE2006F08C900831603133F08F0004008F10092
:101DF2004108F2000A168A15A4260A128A157008EA
:101E020083120313CA007108CB007208CC000A16B1
:101E12008A11F7260A128A158312031347088316BA
:101E22000313B40083120313480883160313B50087
:101E32008312031349084E2F023083126B06031DCF
:101E4200512F831603133F0883120313A70083162F
:101E52000313400883120313A800831603134108D7
:101E620083120313A9006D08AA006E08AB006F0865
:101E7200AC000A168A1150250A128A15831203131E
:101E8200270883160313B40083120313280883164A
:101E92000313B50083120313290883160313722F49
:101EA200033083126B06031D732F831603133F083F
:101EB200F8004008F9004108FA00831203136D0884
:101EC200FB006E08FC006F08FD000A168A11D7237A
:101ED2000A128A15780883160313B4007908B5002C
:101EE2007A08B6008312E901073069020318892FC4
:101EF2002030E4006908903E840064088317800063
:101F02000130E4006408E90707306902031C792FF5
:101F12009430E4006408DA00831603133408831251
:101F22000313DB0083160313350883120313DC004B
:101F320083160313360883120313DD0090300A124E
:101F42008A11A0210A128A15023083120313E400B7
:101F52006408FA009030FB000130FC0001300A16E0
:101F62008A11F4200A128A15003083160313B40072
:101F72000030B5000030B60083120313E701E70A10
:101F820001308312E4006408EA07831603133D0359
:101F9200031D4A2CBD0183120313EA0114306A02A5
:101FA2000318E02F6A08A03E8400831380010130E9
:101FB200E4006408EA0714306A02031CD32FFA0112
:101FC200FA0A7730FB008030FC0001300A168A11D1
:101FD200F4200A128A15023083120313E400640803
:101FE200FA007730FB008030FC0001300A168A11BB
:101FF200F4200A128A1583120313EA014A2CFF1BEA
:102002000A2883137F1883170008840A0319FF0A1A
:10201200080010308A000408840A82070034013460
:102022000034003400340A340034003400346434A0
:10203200003400340034E834033400340034103403
:10204200273400340034A034863401340034403460
:1020520042340F34003480349634983400340034DF
:10206200E134F53405340034CA349A343B34003454
:1020720080343F340034203441340034C834423494
:1020820000347A34443440341C3446345034C3343B
:102092004734243474344934973418344B34BC34C0
:1020A200BE344C346B346E344E34033415345034F5
:1020B2007934AD346034F3344934713400348034CB
:1020C2003F34CD34CC343D34D73423343C34123411
:1020D20083343A34B734D1343834C63427343734BD
:1020E200383486343534C034D6343334CC342B349B
:1020F2003234703489343034E734DB342E34E5340E
:102102003C341E344234A2340D3420342034203482
:10211200203420342034203420342034203420341D
:1021220020342034203420340034433441344C34BD
:10213200433455344C3441345434523449344334A6
:0E2142004534003425342E34353466340034F0
:1021520083120313A600A501261CB3282408FC0041
:102162007C08A5070310A40D0310A60C2608031D66
:10217200AD2825080800F9001930F0000030F10000
:102182000A168A15D0260A168A11E5287908803E91
:102192000A168A155A2708007908C03E0A168A15B7
:1021A2005A2708007908943E0A168A155A27080009
:1021B2007908D43E0A168A155A2708007908803E03
:1021C2000A168A155A2708007808013A0319C728FF
:1021D200033A0319CD28013A0319D328073A031900
:1021E200D928DF28080083120313A000A101A2014D
:1021F2007A08FD007D08F80020080A168A11BC2022
:102202000A168A118312031321087B0784007C08B3
:1022120003187C0AFF000A168A1100200A168A1186
:10222200003A031908008312031321087B07840074
:102232007C0803187C0AFF000A168A1100200A167D
:102242008A110A168A1582270A168A110130831208
:102252000313A1070318A20A0030A2070329F601FB
:10226200F31F3A29F209F309F20A0319F30AF601F4
:10227200F60AF11F4129F009F109F00A0319F10ADE
:102282007008710403196E29F501F50AF11B55292D
:1022920001300310F00DF10DFF3E031D4A290130FC
:1022A200F4007408F507472971087302031D5B29BE
:1022B20070087202031C63297008F2027108031C81
:1022C200F303F30201300310F10CF00CFF3E031D87
:1022D20064290130F502031D552976080319762970
:1022E200F209F309F20A0319F30A7308F1007208FA
:1022F200F000080073087204710470040319BE2907
:10230200F901F90AF31B93290130F8000310F00DCB
:10231200F10DF20DF30DF80B87290130F800780862
:10232200F907832973087702031DA129720876022F
:10233200031DA12971087502031DA12970087402E9
:10234200031CB1297008F4027108031C710FF50215
:102352007208031C720FF6027308031C730FF70254
:1023620001300310F30CF20CF10CF00CFF3E031DD4
:10237200B2290130F902031D93297708F300760888
:10238200F2007508F1007408F000080083120313CC
:10239200A101F81FD329F709F809F70A0319F80A66
:1023A200A101A10AFA1FDE29F909FA09F90A03199A
:1023B200FA0A0130FB007B08A106A201A3017708FB
:1023C20078040319152AA001A00AF81BF429013088
:1023D2000310F70DF80DFF3E031DE9290130FB0044
:1023E2007B08A007E62901300310A20DA30DFF3ED2
:1023F200031DF52978087A02031D012A770879025C
:10240200031C0A2A7708F9027808031CFA03FA0265
:10241200221401300310F80CF70CFF3E031D0B2AA7
:102422000130A002031DF429210803191D2AA20963
:10243200A309A20A0319A30A2308F8002208F70035
:102442000800F21F492A0030F6000030F700803001
:10245200F8007009F9007109FA007209FB00F90A23
:102462000319FA0A0319FB0A7908F6077A0803180E
:102472007A0F3C2A3D2AF7077B0803187B0F422A72
:10248200432AF8077608F0007708F1007808F2008E
:10249200F51F702A0030F6000030F7008030F80097
:1024A2007309F9007409FA007509FB00F90A0319A6
:1024B200FA0A0319FB0A7908F6077A0803187A0F51
:1024C200632A642AF7077B0803187B0F692A6A2AA2
:1024D200F8077608F3007708F4007808F5008030F2
:1024E200F2068030F50675087202031D08007408B2
:1024F2007102031D08007308700208000030FC001E
:102502000030FB000030FA000030F900730872045A
:10251200710470040319D42AFD01FD0AF31B9F2ADA
:102522000130F8000310F00DF10DF20DF30DF80B70
:10253200932A0130F8007808FD078F2A0130F8004D
:102542000310F90DFA0DFB0DFC0DF80BA12A73080F
:102552007702031DB62A72087602031DB62A710895
:102562007502031DB62A70087402031CC72A70087C
:10257200F4027108031C710FF5027208031C720F3A
:10258200F6027308031C730FF7027914013003106B
:10259200F30CF20CF10CF00CFF3E031DC82A0130C3
:1025A200FD02031D9F2A7C08F3007B08F2007A08D3
:1025B200F1007908F000080073080319E52A72088F
:1025C20071047004031DF82A0030F0000030F1009D
:1025D2000030F20008000130F5007508F307013001
:1025E2000310F20CF10CF00CFF3E031DF12AFE3039
:1025F20072050319132BEC2A0130F5007508F30755
:102602000130F007003003180130F10700300318E1
:102612000130F20701300310F20CF10CF00CFF3E16
:10262200031D0C2BFF3072050319222BFD2A0130EA
:10263200F30201300310F00DF10DF20DFF3E031D08
:102642001B2BF11B282B023073020318182B731853
:10265200302BFF30F0057F30F105FF30F20503101B
:10266200F30C7308F500F601F70110300310F50DB5
:10267200F60DF70DFF3E031D372B7508F0047608A3
:10268200F1047708F204740803190800F21708002D
:10269200831203134008C4004108C5004208C60063
:1026A2000310450D460DC7004708CD004D08031D18
:1026B200632B0030C3000030C2000030C100003084
:1026C200C00008004008C4004108C5004208C60016
:1026D20017300310C60CC50CC40CFF3E031D6A2B39
:1026E2004408C7004708C800C117FF30C005FF30C3
:1026F200C1050030C2054008C9004108CA004208AD
:10270200CB00CC018E30CD02CD1FA52B4D08803AD7
:102712008F3E0318952B0030C3000030C2000030FA
:10272200C1000030C000080001300310CC0CCB0CFB
:10273200CA0CC90CFF3E031D962B0130C40044088D
:10274200CD070319C02B952B18304D02031CBD2B4E
:102752000030C3000030C2000030C1000030C000B1
:1027620008000130C4000310C90DCA0DCB0DCC0DF9
:10277200C40BB42B0130CD024D08031DB22B480807
:102782000319CE2BC909CA09CB09CC09C90A0319F5
:10279200CA0A0319CB0A0319CC0A4C08C3004B0816
:1027A200C2004A08C1004908C00008007B08831221
:1027B2000313A0007C08A1007D08A2000310210DD4
:1027C200220DA3002308A8002808031DEF2B0030C8
:1027D200F8000030F9000030FA0008007808A00084
:1027E2007908A1007A08A2000310210D220DA3008E
:1027F2002308A9002908031D052C0030F800003029
:10280200F9000030FA0008000030A5000030A600F0
:102812000030A70089302907A0002008A8027B0801
:10282200A0007C08A1007D08A20010300310A20CB9
:10283200A10CA00CFF3E031D172C2008A3002308A7
:10284200A9007808A0007908A1007A08A200103037
:102852000310A20CA10CA00CFF3E031D292C200882
:10286200A3002308A9068030A0002008A905FC17B0
:10287200FF30FB05FF30FC050030FD05F917FF3086
:10288200F805FF30F9050030FA051830A0002008DD
:10289200A40001300310A50DA60DA70DFF3E031DD8
:1028A2004B2C7A087D02031D5C2C79087C02031DE7
:1028B2005C2C78087B02031C692C7808FB027908DF
:1028C200031C790FFC027A08031C7A0AFD02251404
:1028D20001300310FB0DFC0DFD0DFF3E031D6A2CA4
:1028E2000130A402031D4A2C2508F0002608F1003D
:1028F2002708F2002808A0002008F3002908A100F8
:102902002108F4000A168A11DD227008F800710805
:10291200F9007208FA0008007008F6007108F70062
:102922007208F8000310770D780DF9007908831208
:102932000313A5002508031DA72C0030F300003067
:10294200F2000030F1000030F00008007308F600D9
:102952007408F7007508F8000310770D780DF90078
:102962007908A4002408031DBF2C0030F3000030B6
:10297200F2000030F1000030F0000800F117FF30E3
:10298200F005FF30F1050030F205F417FF30F305D2
:10299200FF30F4050030F5050030A3000030A2003E
:1029A2000030A1000030A0007F30A502983024073B
:1029B200F6007608A5021830F6007608A400013069
:1029C200F6000310A00DA10DA20DA30DF60BE22C33
:1029D20075087202031DF32C74087102031DF32C97
:1029E20073087002031C002D7308F0027408031CA4
:1029F200740FF1027508031C750AF20220140130EB
:102A02000310F00DF10DF20DFF3E031D012D0130FB
:102A1200A402031DE02CA51F2C2D2508803A973E09
:102A220003181C2D0030F3000030F2000030F100DA
:102A32000030F000080001300310A30CA20CA10C1E
:102A4200A00CFF3E031D1D2D0130F6007608A507E0
:102A52000319472D1C2D18302502031C442D00306C
:102A6200F3000030F2000030F1000030F000080006
:102A72000130F6000310A00DA10DA20DA30DF60B5F
:102A82003B2D0130A5022508031D392D2308F30033
:102A92002208F2002108F1002008F0000800831249
:102AA20003132708AD002808AE002908AF00031061
:102AB2002E0D2F0DB0003008B1003108031D682D16
:102AC2000030A7000030A8000030A90008002A0842
:102AD200AD002B08AE002C08AF0003102E0D2F0DF9
:102AE200B0003008B6003608031D7E2D0030A70066
:102AF2000030A8000030A900080036087B3EAD0077
:102B02002D08B1072708AD002808AE002908AF003C
:102B120010300310AF0CAE0CAD0CFF3E031D8A2D1E
:102B22002D08B0003008B6002A08AD002B08AE0010
:102B32002C08AF0010300310AF0CAE0CAD0CFF3EF2
:102B4200031D9C2D2D08B0003008B6068030AD0064
:102B52002D08B605A817AB17FF30AA05FF30AB0545
:102B62000030AC050030B2000030B3000030B400D9
:102B72000730AD002D08B500271CCD2D2A08B2075D
:102B82002B08031103182B0A031DB3072C0803118A
:102B920003182C0A031DB40701300310A90CA80C5A
:102BA200A70CFF3E031DCE2D01300310AA0DAB0D65
:102BB200AC0DFF3E031DD62D0130B502031DBD2D08
:102BC2000930AD002D08B500271CF52D2A08B207E3
:102BD2002B08031103182B0A031DB3072C0803113A
:102BE20003182C0A031DB40701300310A90CA80C0A
:102BF200A70CFF3E031DF62D01300310B40CB30CDD
:102C0200B20CFF3E031DFE2D0130B502031DE52D62
:102C12003208F0003308F1003408F2003108AD0048
:102C22002D08F3003608AE002E08F4000A168A11A9
:102C3200DD22700883120313A7007108A80072082E
:102C4200A9000800F901831203130816081C2C2E90
:102C5200F901F90A3A2E881C302E0230372E081D4F
:102C6200342E0330372E881D3A2E0430F0007008BF
:102C7200F9000812F101F2017208803AFF00803077
:102C82007F02031D462E0A3071020318592E0130AD
:102C9200F1070318F20A0030F2077208803AFF00C7
:102CA20080307F02031D572E0A307102031C482E0A
:102CB200831203138816081C602E05306B2E881CA5
:102CC200642E06306B2E081D682E07306B2E881D71
:102CD2006E2E0830F0007008F9008812F301F4013A
:102CE2007408803AFF0080307F02031D7A2E0A307A
:102CF200730203188D2E0130F3070318F40A003013
:102D0200F4077408803AFF0080307F02031D8B2E87
:102D12000A307302031C7C2E831203130817081C4B
:102D2200942E09309F2E881C982E0A309F2E081D43
:102D32009C2E0B309F2E881DA22E0C30F0007008A6
:102D4200F9000813F501F6017608803AFF00803099
:102D52007F02031DAE2E0A3075020318C12E013008
:102D6200F5070318F60A0030F6077608803AFF00E6
:102D720080307F02031DBF2E0A307502031CB02E65
:102D8200831203138817081CC82E0D30D32E881CFB
:102D9200CC2E0E30D32E081DD02E0F30D32E881DF0
:102DA200D62E1030F0007008F9008813F701F801F0
:102DB2007808803AFF0080307F02031DE22E0A303D
:102DC20077020318F52E0130F7070318F80A0030CE
:102DD200F8077808803AFF0080307F02031DF32E47
:102DE2000A307702031CE42E7908080083120313C9
:102DF2004708CD004808CE004908CF0003104E0D09
:102E02004F0DD0005008D3004A08CD004B08CE0029
:102E12004C08CF0003104E0D4F0DD0005008D200C9
:102E220053080319202F520853020318272F530364
:102E3200FF3A5207CD0019304D02031C272F4A08D2
:102E4200C7004B08C8004C08C90008005208031903
:102E52000800530852020318362F5203FF3A530751
:102E6200CD0019304D02031808000630CD004D0880
:102E7200D100C91BD117CC1B5117C817FF30C7058A
:102E8200FF30C8050030C905CB17FF30CA05FF3037
:102E9200CB050030CC05520853020318762F0130BF
:102EA2000310CA0DCB0DCC0DFF3E031D512F013077
:102EB200D202520853060319712F0130D102510870
:102EC20007390319712F502F01300310C90CC80C98
:102ED200C70CFF3E031D662F0130CD004D08D307FE
:102EE2005308520603199F2F652F530852020318E5
:102EF2009F2F01300310C70DC80DC90DFF3E031DE2
:102F02007B2F0130D3025208530603199B2F013045
:102F1200D1025108073903199B2F7A2F0130031070
:102F2200CC0CCB0CCA0CFF3E031D902F0130CD0000
:102F32004D08D20753085206031D8F2FD11FB12F00
:102F4200FF30C706FF30C806FF30C9060130C70789
:102F5200003003180130C807003003180130C907D8
:102F6200511FC32FFF30CA06FF30CB06FF30CC06FD
:102F72000130CA07003003180130CB0700300318B4
:102F82000130CC07D1014708CA07480803110318CA
:102F9200480A031DCB07490803110318490A031DF8
:102FA200CC07CC1FE62FFF30CA06FF30CB06FF301E
:102FB200CC060130CA07003003180130CB070030BD
:102FC20003180130CC07D101D10A4A08F0004B089E
:102FD200F1004C08F2005308CD004D08F3005108EF
:102FE200CE004E08F4000A168A11DD227008831200
:0E2FF2000313C7007108C8007208C900080068
:103D3E0001300A168A155A27080072087104700499
:103D4E00031908008030F206080064008001840A1E
:103D5E000406031900340406AD2EF100F0013A30CA
:103D6E0071020318C02E30307102031CC02EF001F8
:103D7E00F00A700C08007008F4007108F500720863
:103D8E00F300740884008317751C83137308800076
:103D9E000800831603133A087102031DD82E390842
:103DAE007002031CE32E013083160313B9070318A8
:103DBE00BA0A0030BA07D02EB901BA01080083162C
:103DCE000317880189018312031787018801F030D8
:103DDE00831603138500860187010F308800083093
:103DEE0089000A128A1501200800FB007B08831245
:103DFE000313A000A101A2012008F0002108F10088
:103E0E002208F2008E30A3002308F300F4010A16F4
:103E1E008A11DD227008F8007108F9007208FA00A4
:103E2E000800831203135608550454040319212F56
:103E3E008030D6065708C7005808C8005908C90070
:103E4E005408CA005508CB005608CC000A168A1131
:103E5E00F726831203134708D4004808D5004908F3
:103E6E00D6000800F401F501701C432F7208F40708
:103E7E000318F50A7308F50701300310F20DF30D60
:103E8E00FF3E031D442F01300310F10CF00CFF3EDA
:103E9E00031D4B2F70087104031D3B2F7508F10095
:103EAE007408F0000800F700831203130713143090
:103EBE00F0000030F1000A168A15D0260A168A156F
:103ECE000630F0000030F1007708F6007608F200B8
:103EDE000A168A15C2260A168A1583120313871725
:103EEE001430F0000030F1000A168A15D026831225
:103EFE00031387130800F70083120313071702300A
:103F0E00F0000030F1000A168A15D0260A168A151E
:103F1E000630F0000030F1007708F6007608F20067
:103F2E000A168A15C2260A168A15831203138717D4
:103F3E000230F0000030F1000A168A15D0268312E6
:103F4E00031387130800FC01FB010A168A112326AE
:103F5E000A168A15FA007A08FC007C0883160313E9
:103F6E003B060319D32FE830F0000330F1000A1698
:103F7E008A15D0260A168A157C08FA007A08831646
:103F8E000313BB007C080319D12F7C08FA007A08B2
:103F9E00FB000800FB010800FB0108008E30FC004E
:103FAE007C08FD00FF307B050319EB2F0130031059
:103FBE00FB0CFA0CF90CF80CFF3E031DDE2F013042
:103FCE00FC007C08FD07D92F7808F0007908F10075
:103FDE007A08F2007D08FC007C08F300F4010A1652
:103FEE008A11DD227008F8007108F9007208FA00D3
:023FFE000800B9
:04400E00D4E0FFFEFD
:00000001FF
